:100000000C942A001895000018950000189500001F
:10001000189500001895000018950000189500002C
:100020001895000018950000189500000C94DA014E
:10003000189500000C9412120C94441218950000AC
:1000400018950000189500001895000018950000FC
:10005000189500008FE58DBFCCEFECE44E2E88E0C4
:100060008EBFD7E0F7E05F2EEEEFF7E0A0E6B0E05E
:10007000A89584B7082E877F84BF88E1992781BD22
:1000800091BD88278D933197E9F780E189B980E0A8
:1000900080BD88E18AB96624579A0E94271384B7E5
:1000A000877F84BF88E181BD80E081BD80E08ABB1D
:1000B0008CE187BB83EE88BB80E084BB8FEF85BB80
:1000C00080EF81BB8FE082BB87E886B980E087B98B
:1000D000379A85E083BF81EB8FBD81E08EBD8FEFC6
:1000E0008ABDA4ECB1E0E8E5F6E20E945E10A6EC61
:1000F000B1E0EAE5F6E20E945E108FEF8ABD80E093
:1001000088BD0CEF13E020E030E0AFEEB0E00D93DF
:100110001D932D933C9380E080931F01C29A86E942
:1001200090E00E942C10C39A86E990E00E942C1067
:10013000C49A8AEF90E00E942C10C298C398C49889
:1001400080E090E0A5EEB0E08D939C9301E010E09C
:1001500020E030E0ABEFB0E00D931D932D933C9386
:100160004AE050E060E070E0ABEFB0E00D911D912F
:100170002D913C910E9475121CF011F00C94E0003E
:10018000A5EEB0E00D911C910F931F9307B1007E77
:10019000076007B90E946410482F592F1F910F91D3
:1001A000040F151FA5EEB0E00D931C9381E090E0C5
:1001B0000E942C10ABEFB0E00E94DB0E0C94B0005C
:1001C000A5EEB0E00D911C914AE050E00E94FB0EBC
:1001D000A5EEB0E04D935C9382E090E00E942C107D
:1001E000A5EEB0E00D911C91043650E015070CF41B
:1001F00002C00C94000184E0809334010C94640CE0
:100200000E942B0A789489B7816089BF0091BA0156
:10021000013011F00C943A0180E08093BA01A5E31B
:10022000B1E03FE30E94440FA5E3B1E08C91082FB9
:100230000A3011F00C943801A5E3B1E00E942113BB
:10024000082F41E0041BABEBB1E00C93A5E3B1E058
:100250000E942113EA2FFB2F0091BB013197E01B75
:10026000F10B0FEFA5E3B1E00E9419130C941401F8
:100270000E94A00C87E090E00E942C10ECE5F6E2D2
:100280000E94890FA4E3B7E0E3E0F1E00E948B1243
:100290000E94810F0E94900F87E090E00E942C1036
:1002A000E2E6F6E20E94890FA4E3B7E0E0E7F0E0BF
:1002B0000E948B120E94810F0E94900F87E090E0B5
:1002C0000E942C10E8E6F6E20E94890FA4E3B7E052
:1002D000E2E3F1E00E9488120E94810F0E94900FD9
:1002E00087E090E00E942C10EEE6F6E20E94890F73
:1002F000A4E3B7E0E0E3F1E00E9488120E94810FDE
:100300000E94900F87E090E00E942C10E4E7F6E254
:100310000E94890FA4E3B7E0E0E2F1E00E948B12B3
:100320000E94810F0E94900F87E090E00E942C10A5
:10033000EAE7F6E20E94890FA4E3B7E0EBE0F1E020
:100340000E948B120E94810F0E94900F87E090E024
:100350000E942C10E0E8F6E20E94890FA4E3B7E0C7
:10036000E7E0F1E00E9490120E94810F0E94900F3E
:1003700087E090E00E942C10E6E8F6E20E94890FE8
:10038000A4E3B7E0E9E0F1E00E9490120E94810F3F
:100390000E94900F87E090E00E942C10ECE8F6E2BB
:1003A0000E94890FE2E9F6E20E94890F0E94900FF5
:1003B0000C9406010F921F922F923F924F925F92E0
:1003C0007F92AF92BF920F931F932F933F934F93C0
:1003D0005F936F937F938F939F93AF93BF93CF93CD
:1003E000DF93EF93FF938FB78F93A89584E6809365
:1003F00052000E9423020E94C4030E9419050E9419
:10040000D6050E9409070E94C8080E949E098F9184
:100410008FBFFF91EF91DF91CF91BF91AF919F91EE
:100420008F917F916F915F914F913F912F911F918C
:100430000F91BF90AF907F905F904F903F902F9023
:100440001F900F90189507B1007E056007B90E94B4
:100450006410AFEDB0E08D939D9388278D938C93BE
:1004600000E014E020E030E0AFEDB0E04D915D91B0
:100470006D917C910E947012AFEDB0E00D931D93D1
:100480002D933D9307B1007E036007B90E9464106D
:10049000ABEDB0E08D939D9388278D938C9307B13E
:1004A000007E006007B90E946410A3EEB0E08D9357
:1004B0009C9307B1007E066007B90E946410A4E215
:1004C000B1E08D939C9300E014E00F931F9307B16C
:1004D000007E076007B90E946410482F592F1F91B2
:1004E0000F91041B150BA5EEB0E00D931C93ABED23
:1004F000B0E00D911D912D913C914AE050E060E0FB
:1005000070E00E943B10ABEDB0E00D931D932D9376
:100510003D93AFEDB0E00D911D912D913C914AE0DE
:1005200050E060E070E00E943B10AFEDB0E00D9352
:100530001D932D933D93A7EEB0E00D911D912D914C
:100540003C914AEF50E060E070E00E94C40FABEFD6
:10055000B0E04D935D936D937D93A7EEB0E00D9168
:100560001D912D913C91ABEFB0E04D915D916D915E
:100570007C910E947012A7EEB0E00D931D932D9315
:100580003D93ABEDB0E00D911D912D913C91A0E319
:10059000B1E04D915C91662777270E947012ABEF16
:1005A000B0E00D931D932D933D93A7EEB0E00D9118
:1005B0001D912D913C91ABEFB0E04D915D916D910E
:1005C0007C910E946B12A7EEB0E00D931D932D93CA
:1005D0003D93ABEEB0E00D911D912D913C914AEF12
:1005E00050E060E070E00E94C40FA7EFB0E04D93D0
:1005F0005D936D937D93ABEEB0E00D911D912D91C8
:100600003C91A7EFB0E04D915D916D917C910E947E
:100610007012ABEEB0E00D931D932D933D93ABEEB6
:10062000B0E00D911D912D913C91AFEDB0E04D9159
:100630005D916D917C910E946B12ABEEB0E00D93D9
:100640001D932D933D93ABEEB0E00D911D912D9137
:100650003C9149E150E060E070E00E94C40FA7EFD8
:10066000B0E04D935D936D937D93AFEDB0E00D9150
:100670001D912D913C914AE050E060E070E00E94B5
:100680003B10ABEFB0E00D931D932D933D93A7EF7F
:10069000B0E00D911D912D913C91ABEFB0E04D91EB
:1006A0005D916D917C910E947012A7EFB0E00D9367
:1006B0001D932D933D93A7EFB0E00D911D912D91CA
:1006C0003C9143E250E060E070E00E943B10A7EFF5
:1006D000B0E00D931D932D933D93A7EFB0E00D91E6
:1006E0001D912D913C9144E650E060E070E00E9445
:1006F000C40FA7E1B1E04D935D936D937D93A7EE99
:10070000B0E00D911D912D913C91A7E1B1E04D918B
:100710005D916D917C910E946B12A7EEB0E00D93FC
:100720001D932D933D930AEF10E020E030E0ABEFF6
:10073000B0E00D931D932D933C93A7EEB0E00D9187
:100740001D912D913C91ABEFB0E04D915D916D917C
:100750007C910E94C40FA3E0B1E04D935D936D9333
:100760007D93A7E1B1E00D911D912D913C914AE05F
:1007700050E060E070E00E94C40FA7E1B1E04D934B
:100780005D936D937D93089507B1007E046007B972
:100790000E946410A4E6B0E08D939D9388278D930A
:1007A0008C9307B1007E026007B90E946410A0E636
:1007B000B0E08D939D9388278D938C93A0E6B0E055
:1007C0000D911D912D913C914AE050E060E070E068
:1007D0000E943B10A0E6B0E00D931D932D933D9336
:1007E000A4E6B0E00D911D912D913C914AE050E0BE
:1007F00060E070E00E943B10A4E6B0E00D931D9312
:100800002D933D93A8E6B0E00D911D912D913C9163
:100810004AEF50E060E070E00E94C40FA8E7B0E04B
:100820004D935D936D937D93A8E6B0E00D911D917E
:100830002D913C91A8E7B0E04D915D916D917C9137
:100840000E947012A8E6B0E00D931D932D933D9386
:10085000A0E6B0E00D911D912D913C91ACE7B0E088
:100860004D915C91662777270E947012A8E7B0E04F
:100870000D931D932D933D93A8E6B0E00D911D912E
:100880002D913C91A8E7B0E04D915D916D917C91E7
:100890000E946B12A8E6B0E00D931D932D933D933B
:1008A000ACE6B0E00D911D912D913C914AEF50E0E6
:1008B00060E070E00E94C40FA7EFB0E04D935D933D
:1008C0006D937D93ACE6B0E00D911D912D913C911F
:1008D000A7EFB0E04D915D916D917C910E947012F7
:1008E000ACE6B0E00D931D932D933D93ACE6B0E0E4
:1008F0000D911D912D913C91A4E6B0E04D915D913B
:100900006D917C910E946B12ACE6B0E00D931D934B
:100910002D933D93ACE6B0E00D911D912D913C914E
:1009200049E150E060E070E00E94C40FA7EFB0E042
:100930004D935D936D937D93A4E6B0E00D911D9171
:100940002D913C914AE050E060E070E00E943B1045
:10095000ABEFB0E00D931D932D933D93A7EFB0E067
:100960000D911D912D913C91ABEFB0E04D915D91BA
:100970006D917C910E947012A7EFB0E00D931D93D2
:100980002D933D93A7EFB0E00D911D912D913C91DA
:1009900043E250E060E070E00E943B10A7EFB0E05F
:1009A0000D931D932D933D93A7EFB0E00D911D91F5
:1009B0002D913C9144E650E060E070E00E94C40F4D
:1009C000A4E7B0E04D935D936D937D93A8E6B0E00E
:1009D0000D911D912D913C91A4E7B0E04D915D9159
:1009E0006D917C910E946B12A8E6B0E00D931D936F
:1009F0002D933D930AEF10E020E030E0ABEFB0E044
:100A00000D931D932D933C93A8E6B0E00D911D919D
:100A10002D913C91ABEFB0E04D915D916D917C914A
:100A20000E94C40FA0E7B0E04D935D936D937D935A
:100A30000895A3E0B1E00D911D912D913C91A3E1AA
:100A4000B1E04D915D916D917C910E946B12ABE193
:100A5000B1E00D931D932D933D93A7E1B1E00D916E
:100A60001D912D913C91ABE1B1E04D915D916D9166
:100A70007C910E946B12ABE1B1E00D931D932D931D
:100A80003D93ABE1B1E00D911D912D913C9141E180
:100A900050E060E070E00E943B10ABE1B1E00D93EC
:100AA0001D932D933D93A0E2B1E00D911D912D91E9
:100AB0003C91ABE1B1E04D915D916D917C910E94D3
:100AC0006B12A0E2B1E00D931D932D933D9348ED81
:100AD00056ED60E070E0A0E2B1E00D911D912D9126
:100AE0003C910E9475121CF011F00C9479050C9445
:100AF000830508ED16ED20E030E0A0E2B1E00D93B3
:100B00001D932D933C9348E259E26FEF7FEFA0E2F3
:100B1000B1E00D911D912D913C910E9475120CF444
:100B200002C00C949D0508E219E22FEF3FEFA0E20E
:100B3000B1E00D931D932D933C93A0E2B1E00D9194
:100B40001D912D913C914BE950E060E070E00E94D6
:100B5000C40FABEFB0E04D935D936D937D93ABE12C
:100B6000B1E00D911D912D913C9145EA50E060E07E
:100B700070E00E94C40FA7EFB0E04D935D936D93BA
:100B80007D93ABEFB0E00D911D912D913C91A7EFBE
:100B9000B0E04D915D916D917C910E946B12ABE044
:100BA000B1E00D931D932D933D930895AEE2B1E016
:100BB0000D911D9117FB1EF42FEF3FEF02C022276E
:100BC0003327A4E2B1E04D915D9157FB1EF46FEF26
:100BD0007FEF02C0662777270E947012AAE2B1E079
:100BE0000D931D932D933D93A0E2B1E00D911D91C6
:100BF0002D913C9140E25EE460E070E00E94C40F01
:100C0000A7EFB0E04D935D936D937D93A7EFB0E0B8
:100C10000D911D912D913C910E941810A7EFB0E00D
:100C20000D931D932D933D9341E050E060E070E003
:100C3000A7EFB0E00D911D912D913C910E9475128E
:100C40000CF402C00C942E0601E010E020E030E02D
:100C5000A7EFB0E00D931D932D933C93AAE2B1E072
:100C60000D911D912D913C91A7EFB0E04D915D91BB
:100C70006D917C910E94C40FAAE2B1E04D935D9307
:100C80006D937D93A0E2B1E00D911D912D913C916A
:100C900040ED57E060E070E00E94C40FA7EFB0E0C5
:100CA0004D935D936D937D93A7EFB0E00D911D91F2
:100CB0002D913C910E941810A7EFB0E00D931D9369
:100CC0002D933D9346E150E060E070E0A7EFB0E087
:100CD0000D911D912D913C910E9475121CF011F007
:100CE0000C9474060C947E0606E110E020E030E0DF
:100CF000A7EFB0E00D931D932D933C930BE110E013
:100D000020E030E0A7EFB0E04D915D916D917C91D6
:100D10000E947012A7EFB0E00D931D932D933D93A9
:100D2000A7EFB0E00D911D912D913C914FEF5FEF3A
:100D30006FEF7FEF0E943B10AFEFB0E00D931D937C
:100D40002D933D93A7EFB0E04D915D916D917C9116
:100D5000AAE2B1E00D911D912D913C910E94751276
:100D60001CF011F00C94B6060C94C206A7EFB0E08C
:100D70000D911D912D913C91AAE2B1E00D931D932F
:100D80002D933C93AFEFB0E04D915D916D917C91CF
:100D9000AAE2B1E00D911D912D913C910E94751236
:100DA0000CF402C00C94E006AFEFB0E00D911D9181
:100DB0002D913C91AAE2B1E00D931D932D933C93AC
:100DC000AAE2B1E00D911D912D913C91AFE0B1E00F
:100DD0000D931D932D933C93ABE0B1E00D911C91CD
:100DE000AFE0B1E04D915C91041B150BA7E0B1E0C1
:100DF0000D931C93ABE0B1E00D911C91AFE0B1E01D
:100E00004D915C91040F151FA9E0B1E00D931C9367
:100E1000089500911F01003011F00C94750780E0D7
:100E200090E0A7E0B1E08D939C9380E090E0A9E092
:100E3000B1E08D939C9300E010E020E030E0ABE067
:100E4000B1E00D931D932D933C9300E010E020E062
:100E500030E0A3E1B1E00D931D932D933C9300E0AE
:100E600010E020E030E0A0E2B1E00D931D932D935F
:100E70003C9300E010E020E030E0A3E0B1E00D930F
:100E80001D932D933C9300E010E020E030E0A7EEAE
:100E9000B0E00D931D932D933C9300E010E020E013
:100EA00030E0A6E2B1E00D931D932D933C93A5EEA7
:100EB000B0E00D911C91023350E015071CF011F0C9
:100EC0000C9464070C9473070E942B0A81E08093B2
:100ED0001F0100E010E020E030E0A6E2B1E00D9359
:100EE0001D932D933C930C94C708013011F00C9482
:100EF0002608A5EEB0E00D911C91023350E01507D5
:100F00000CF402C00C942408A6E2B1E00E94DB0EAF
:100F100043E050E060E070E0ABE0B1E00D911D9186
:100F20002D913C910E94751280E014F009F081E04F
:100F30008F9344E650E060E070E0A6E2B1E00D91EE
:100F40001D912D913C910E94751280E00CF481E07E
:100F50009F918923882311F40C94D407ABE0B1E06E
:100F60004D915D916D917C91A3E1B1E00D911D9149
:100F70002D913C910E9475120CF402C00C94D20782
:100F8000A3E1B1E00D911D912D913C9142E050E023
:100F900060E070E00E946B12A3E1B1E00D931D933D
:100FA0002D933D930C9424084DEF5FEF6FEF7FEF8F
:100FB000ABE0B1E00D911D912D913C910E94751215
:100FC00080E00CF481E08F9344E650E060E070E054
:100FD000A6E2B1E00D911D912D913C910E947512F8
:100FE00080E00CF481E09F918923882311F40C9414
:100FF0002108ABE0B1E04D915D916D917C91A3E151
:10100000B1E00D911D912D913C910E9475121CF043
:1010100011F00C940D080C941F08A3E1B1E00D91A0
:101020001D912D913C9142E050E060E070E00E9403
:101030007012A3E1B1E00D931D932D933D930C9499
:10104000240883E080931F010C94C708033011F03B
:101050000C94C40881B5886181BD877F81BD00E0A3
:1010600010E020E030E0A6E2B1E00D931D932D9357
:101070003C9301E010E020E030E0A7EFB0E00D93FA
:101080001D932D933C934FEF50E060E070E0A7EF8D
:10109000B0E00D911D912D913C910E9475121CF0B4
:1010A00011F00C94BC08A7E0B1E00D911C91003048
:1010B00050E0150781E009F080E08F93A9E0B1E0EE
:1010C0000D911C91003050E0150781E009F080E09F
:1010D0009F918923882311F40C9470080C94BC0808
:1010E000A7E0B1E00D911C91003050E015071CF015
:1010F00011F00C947D080C948108A7E0B1E00E94E7
:10110000F10EA7E0B1E00D911C91003050E0150701
:101110000CF402C00C949008A7E0B1E00E94EA0E23
:10112000A9E0B1E00D911C91003050E015071CF0D2
:1011300011F00C949D080C94A108A9E0B1E00E9464
:10114000F10EA9E0B1E00D911C91003050E01507BF
:101150000CF402C00C94B008A9E0B1E00E94EA0EC1
:1011600089E190E00E942C100E94C808A7EFB0E02F
:101170000E94DB0E0C94430880E080931F0181B530
:10118000886081BD0C94C70883E080931F01089597
:10119000A7E0B1E00D911C91043B50E015071CF055
:1011A00011F00C94D5080C94DD0884EB90E0A7E0D6
:1011B000B1E08D939C930C94EE08A7E0B1E00D9103
:1011C0001C910C345FEF15070CF402C00C94EE0870
:1011D0008CE49FEFA7E0B1E08D939C93A9E0B1E090
:1011E0000D911C91043B50E015071CF011F00C947C
:1011F000FB080C94030984EB90E0A9E0B1E08D9327
:101200009C930C941409A9E0B1E00D911C910C344D
:101210005FEF15070CF402C00C9414098CE49FEFE7
:10122000A9E0B1E08D939C93A2E3B0E08C9186FBA2
:10123000AAEDB0E08C9185F98C93A2E3B0E08C919B
:1012400087FBAAEDB0E08C9184F98C93A7E0B1E024
:101250000D911C91003050E015070CF402C00C9465
:101260003409969A0C9435099698A9E0B1E00D914D
:101270001C91003050E015070CF402C00C94430997
:10128000979A0C94440997980027AAEDB0E08C91A6
:1012900085FB0EF401E04427A2E3B0E08C9186FBCD
:1012A0000EF44395041711F40C945D098091DA0053
:1012B00080688093DA000C9462098091DA008F775D
:1012C0008093DA000027AAEDB0E08C9184FB0EF445
:1012D00001E04427A2E3B0E08C9187FB0EF4439534
:1012E000041711F40C947B098091DA0080648093D8
:1012F000DA000C9480098091DA008F7B8093DA0009
:10130000A7E0B1E08D919C910E941B0FA3EFB0E08C
:101310008D939C93A9E0B1E08D919C910E941B0F4D
:10132000A5EFB0E08D939C930FEF4091F300041B69
:101330000ABDA5EFB0E08C9188BD0895AFEEB0E096
:101340000D911D912D913C914CE251E060E070E0D7
:101350000E94C40FA7EFB0E04D935D936D937D9312
:10136000AFEEB0E00D911D912D913C91A7EFB0E053
:101370004D915D916D917C910E947012AFEEB0E045
:101380000D931D932D933D93AFEEB0E00D911D9104
:101390002D913C91A3EEB0E04D915D9157FB1EF471
:1013A0006FEF7FEF02C0662777270E946B12AFEEC8
:1013B000B0E00D931D932D933D93AFEEB0E00D91F2
:1013C0001D912D913C914CE251E060E070E00E9453
:1013D000C40FA7EFB0E04D935D936D937D934CEFF9
:1013E00053E060E070E0A7EFB0E00D911D912D910A
:1013F0003C910E9475121CF011F00C94010A0C949F
:10140000040AC29AC398C4984CEF53E060E070E0BD
:10141000A7EFB0E00D911D912D913C910E947512A6
:101420000CF402C00C94170AC39AC498C29840ECFA
:1014300053E060E070E0A7EFB0E00D911D912D91B9
:101440003C910E9475120CF402C00C942A0AC398B5
:10145000C298C49A089581B5886181BD877F81BD96
:1014600080E090E0A4E2B1E08D939C9301E010E075
:1014700020E030E0ABEFB0E00D931D932D933C9353
:101480004AE050E060E070E0ABEFB0E00D911D91FC
:101490002D913C910E9475121CF011F00C94700A71
:1014A000A4E2B1E00D911C910F931F9307B1007E50
:1014B000066007B90E946410482F592F1F910F91A1
:1014C000040F151FA4E2B1E00D931C9381E090E09E
:1014D0000E942C10ABEFB0E00E94DB0E0C94400A8F
:1014E000A4E2B1E00D911C914AE050E00E94FB0E95
:1014F000AEE2B1E04D935C9300E010E020E030E01C
:10150000AFEDB0E00D931D932D933C9301E010E0FF
:1015100020E030E0ABEFB0E00D931D932D933C93B2
:101520004AEF50E060E070E0ABEFB0E00D911D914C
:101530002D913C910E9475121CF011F00C94EF0A51
:1015400007B1007E056007B90E946410A7EFB0E004
:101550008D939D9388278D938C9300E014E020E079
:1015600030E0A7EFB0E04D915D916D917C910E94CC
:101570007012A7EFB0E00D931D932D933D93A7EF4D
:10158000B0E00D911D912D913C914AE050E060E05A
:1015900070E00E943B10A7EFB0E00D931D932D93D8
:1015A0003D93AFEDB0E00D911D912D913C91A7EFD2
:1015B000B0E04D915D916D917C910E946B12AFED09
:1015C000B0E00D931D932D933D9382E090E00E9437
:1015D0002C10ABEFB0E00E94DB0E0C94900AAFED44
:1015E000B0E00D911C914AEF50E00E94210FA2E360
:1015F000B1E04D935C93AFEDB0E00D911D912D9155
:101600003C91ABEEB0E00D931D932D933C9300E025
:1016100010E020E030E0ABEDB0E00D931D932D9392
:101620003C9301E010E020E030E0ABEFB0E00D9340
:101630001D932D933C9344E650E060E070E0ABEFE7
:10164000B0E00D911D912D913C910E9475121CF0FE
:1016500011F00C94560B07B1007E036007B90E948D
:101660006410A7EFB0E08D939D9388278D938C93A2
:10167000ABEDB0E00D911D912D913C91A7EFB0E045
:101680004D915D916D917C910E946B12ABEDB0E03C
:101690000D931D932D933D9382E090E00E942C10BA
:1016A000ABEFB0E00E94DB0E0C941B0BABEDB0E097
:1016B0000D911C914AE050E00E94210FA0E3B1E09F
:1016C0004D935C9300E010E020E030E0A4E6B0E051
:1016D0000D931D932D933C9301E010E020E030E04A
:1016E000ABEFB0E00D931D932D933C934AEF50E088
:1016F00060E070E0ABEFB0E00D911D912D913C9159
:101700000E9475121CF011F00C94C30B07B1007EFF
:10171000046007B90E946410A7EFB0E08D939D9319
:1017200088278D938C93A7EFB0E00D911D912D919B
:101730003C914AE050E060E070E00E943B10A7EF6F
:10174000B0E00D931D932D933D93ACE6B0E00D9169
:101750001D912D913C91A7EFB0E04D915D916D9160
:101760007C910E946B12ACE6B0E00D931D932D931B
:101770003D9382E090E00E942C10ABEFB0E00E941D
:10178000DB0E0C94760B00E010E020E030E0A7EFD9
:10179000B0E00D931D932D933C9301E010E020E009
:1017A00030E0ABEFB0E00D931D932D933C9344E6F6
:1017B00050E060E070E0ABEFB0E00D911D912D9135
:1017C0003C910E9475121CF011F00C94120C07B1A0
:1017D000007E026007B90E946410A0E6B0E08D931D
:1017E0009D9388278D938C93A0E6B0E00D911D9179
:1017F0002D913C91A7EFB0E04D915D916D917C9161
:101800000E946B12A7EFB0E00D931D932D933D93B3
:1018100082E090E00E942C10ABEFB0E00E94DB0E63
:101820000C94D70BA7EFB0E00D911C914AE050E06B
:101830000E94210FACE7B0E04D935C9381B58860C6
:1018400081BDA0E3B1E00D911C91003A5FE0150766
:1018500010F00C94300C83E0809334010C94640CF1
:10186000A0E3B1E00D911C91003757E1150718F086
:1018700011F00C943D0C0C94420C83E080933401E5
:101880000C94640CA2E3B1E00D911C91063950E078
:10189000150710F00C94510C82E0809334010C94E5
:1018A000640CA2E3B1E00D911C910C3251E01507DC
:1018B00018F011F00C945E0C0C94630C82E0809391
:1018C00034010C94640C089581B5886181BD877FD3
:1018D00081BD01E010E020E030E0ABEFB0E00D931F
:1018E0001D932D933C93A4E3B1E04C9155276627BB
:1018F0007727ABEFB0E00D911D912D913C910E94A7
:1019000075121CF011F00C94950CC49A86E990E0C5
:101910000E942C10C49886E990E00E942C10ABEF36
:10192000B0E00E94DB0E0C94730CE2E0F0E00E9449
:10193000BB0F0C94690C089581E08093BA0108955F
:10194000A5E3B1E08C91082F033211F00C94B00C98
:10195000A5E3B1E00E94830F0E94900F0C943D0D0F
:10196000A5E3B1E08C91082F0B3111F00C94C00C61
:10197000A5E3B1E00E94830F0E94900F0C943D0DEF
:10198000A5E3B1E0E8E5F6E22FEF91E00E947210E6
:10199000A3ECB1E00C930091C301003018F011F0FA
:1019A0000C94D40C0C94290DA5E3B1E0EAE9F6E21D
:1019B0002FEF91E00E947210002F003080E010F0B5
:1019C00009F081E08F934091C301A5E3B1E0EAE91A
:1019D000F6E22FEF91E00E947210002F041781E0D1
:1019E00008F080E09F918923882311F40C94040D62
:1019F000A5E3B1E00E94830F0E94900F0E943E0D6C
:101A00000C943D0D0C94270DE5E3F1E00091C3012A
:101A1000A5E7B1E00E941913A5E7B1E00E94E11229
:101A2000ACEBB1E00C930091BC01003011F00C94D0
:101A30001F0D0E943E0D0C943D0D0C94270DA5E347
:101A4000B1E00E94830F0E94900F0C943D0D0C9406
:101A50003D0D0091BC01003011F00C94350D0E9439
:101A60003E0D0C943D0D0C943D0DA5E3B1E00E949C
:101A7000830F0E94900F0C943D0D089581E0809398
:101A8000C901A5E7B1E088278C93A5EBB1E08827D1
:101A90008C93AFEBB1E0E4E5F6E20E940A1280E03D
:101AA00090E0ADEBB1E08D939C93A5E3B1E00E9493
:101AB0002113082F0F93A5E3B1E0E4ECF1E0222716
:101AC00091E00E947210402F0F91041BA3ECB1E033
:101AD0000C93A5E3B1E00E942113EA2FFB2F0091A4
:101AE000C3013197E01BF10B0FEFA5E7B1E00E94B6
:101AF0001913A5EBB1E088278C93A5E7B1E0E6ECDC
:101B0000F1E0222791E00E947210A3ECB1E00C9367
:101B10000091C301003011F00C94950DA5E7B1E0E0
:101B20000E942113A3ECB1E08C9381E08093C80163
:101B30004091C3010091C801041718F011F00C94F2
:101B4000F00D80E3482FA8ECB1E0AD90BB24A4E7F2
:101B5000B1E0AA0DBB1D0C91041781E008F480E0F0
:101B60008F9389E3482FA8ECB1E0AD90BB24A4E7A4
:101B7000B1E0AA0DBB1D0C91041781E010F009F033
:101B800080E09F918923882311F40C94E80DA8EC40
:101B9000B1E0AD90BB24A4E7B1E0AA0DBB1D8C91D0
:101BA000A9ECB1E0AD90BB24A4EBB1E0AA0DBB1D44
:101BB0008C93A9ECB1E08C918F5F8C9380E0A9ECC1
:101BC000B1E0AD90BB24A4EBB1E0AA0DBB1D8C939A
:101BD000A8ECB1E08C918F5F8C9310F40C94980D6D
:101BE000A5EBB1E00E94E112ADEBB1E00D931C93C7
:101BF000A5E7B1E0E6ECF1E0222791E00E94721047
:101C0000002F003018F011F00C94080E0C940F0EF9
:101C10008091DA00877F8093DA000C94140E809113
:101C2000DA0088608093DA00A5E7B1E00E94211312
:101C3000082F0F93A5E7B1E0E6ECF1E0222791E051
:101C40000E947210402F0F91041BA3ECB1E00C9383
:101C5000A5E7B1E00E942113EA2FFB2F0091C301F9
:101C60003197E01BF10B0FEFA5E7B1E00E941913CC
:101C7000A5E7B1E00E943611EDE0F0E0AFEBB1E096
:101C80000E941313ADEBB1E00D911C91013050E0B7
:101C9000150711F00C946A0EA5E3B1E0ECE9F6E249
:101CA0000E945E10A5E3B1E00E943B0FEBEDF0E077
:101CB0000E948B12A5E3B1E00E943B0FE4EAF6E23A
:101CC0000E945E10A5E3B1E00E94830F0E94900F76
:101CD0000C94DA0E023050E0150711F00C948E0EC1
:101CE000A5E3B1E0E6EAF6E20E945E10A5E3B1E00A
:101CF0000E943B0FEFEDF0E00E948B12A5E3B1E0F4
:101D00000E943B0FE4EAF6E20E945E10A5E3B1E018
:101D10000E94830F0E94900F0C94DA0E033050E063
:101D2000150711F00C94AA0EA5E3B1E0EEEAF6E275
:101D30000E945E10A5E3B1E00E943B0FE2E9F6E2EB
:101D40000E945E10A5E3B1E00E94830F0E94900FF5
:101D50000C94DA0E063050E0150711F00C94CE0EFC
:101D6000A5E3B1E0E6EBF6E20E945E10A5E3B1E088
:101D70000E943B0FE3EEF0E00E949012A5E3B1E079
:101D80000E943B0FE4EAF6E20E945E10A5E3B1E098
:101D90000E94830F0E94900F0C94DA0EA5E3B1E02D
:101DA000EEEBF6E20E945E10A5E3B1E00E94830F25
:101DB0000E94900F08950D911D912D913C9181E00D
:101DC000080F8827181F281F381F3C932E931E9337
:101DD0000E930895ED91FC91EF5FFF4FFC93EE930E
:101DE0000895ED91FC91E150F040FC93EE9308953D
:101DF00000FC10D0089503D024D001F8F9CF0024BE
:101E0000E89457FF02C009D0689400F80BD010F88E
:101E10000124089502D009D00895509540954F5F50
:101E20005F4F0895E89417FF0895009510950F5F90
:101E30001F4F6894089599231AF480959095019600
:101E40000895352F242FE894452B11F468940895B4
:101E5000512F402F0027112780E1440F551F001FED
:101E6000111F021B130B416018F4020F131F4E7F4A
:101E70008A9599F708958F938D918823E9F71197A3
:101E80008F910895A4E3B7E018D0883091F08D3099
:101E900039F03323C9F38D933A9563FE44D0F4CFE0
:101EA00063FC04C08DE03FD08AE03DD088278C934E
:101EB000089539D011973395E7CF0F929F93AF9341
:101EC000BF937F938091AE008823E1F3F8948091D3
:101ED000AE008A958093AE009091AC00A4E8B0E08B
:101EE000A90F0024B01D8C919395983209F499277D
:101EF0009093AC0078947F91BF91AF919F910F9098
:101F00000895A4E3B7E08D91882311F00CD0FBCFA6
:101F100008950E943211802D11F005D0FACF089556
:101F20008DE001D08AE09F939FB79F93AF93BF93BB
:101F30000F937F939091D9009832E1F3F8949091A8
:101F4000D90093959093D90099270091D800AFEAD2
:101F5000B0E0A00FB91F8C930395083209F4002755
:101F60000093D800559A7F910F91BF91AF919F91A7
:101F70009FBF9F91089588EE93E06ED03197D9F777
:101F8000089500FC05D0089530D005D001F8F9CFB0
:101F900037D03FD00895842F952FA62FB72FE894E0
:101FA000452B462B472B11F468940895402F512F51
:101FB000622F732F0027112722273327F0E2440FC7
:101FC000551F661F771F001F111F221F331F081B7D
:101FD000190B2A0B3B0B416028F4080F191F2A1F0D
:101FE0003B1F4E7FFA9559F708950024E89477FF38
:101FF00002C006D0689400F809D010F801240895B2
:1020000012D04F5F5F4F6F4F7F4F0895E89437FFB7
:10201000089500951095209530950F5F1F4F2F4F15
:102020003F4F689408954095509560957095089538
:1020300037FF089500951095209530950F5F1F4F3D
:102040002F4F3F4F08953197F1F70895689462F844
:102050000895E89462F80895EF93FF93EE27E82B34
:10206000E92B31F0E0EAFFE03197F1F70197D1F782
:10207000FF91EF9108950F921F922F92C801D901FD
:10208000489F80014A9F90014B9F202C499F100D33
:10209000211D321D5A9F202C589F100D211D321DCD
:1020A000599F200D311D689F200D311D699F300DF6
:1020B000789F300D2F901F900F9008950E9432113D
:1020C0000D920020D9F70895369A3699FECF369AA8
:1020D0003699FECF84B195B1089599910027A90F43
:1020E000B01F1197492F4A955E2F6F2FE894112743
:1020F0004395203019F0C895802D01C08081882338
:10210000B9F07C917723A1F0781739F40EF0042F01
:102110001395689411963196EBCF112321F0411B52
:10212000A11B1127B10BE894E52FF62F1196E0CFF4
:10213000882311F0002708950895D190E190F1903F
:102140000191089521913191419151910895102F5C
:1021500090E8FF0C001F0927990FF7941078652F5E
:1021600090E8440F551F5927990F4795607800381C
:102170000895FF0C90E89027110F9795F794092F79
:102180000895502F2D2D3E2D4F2D612F08952DECAC
:102190003CEC4CEC5DE366270FC0CFDFF2DFDD24C3
:1021A000EE2490E8F92E0FE307C0CCDF05C022270C
:1021B000332740E251E46627552351F1002381F192
:1021C000C6DF71F11627005850580894050B18F413
:1021D00007FD03C025C007FD23C046953795279509
:1021E000F694E794D79422D0FF202AF0DD0CEE1C61
:1021F000FF1C015073F09D2D969548F0DD203AF4B8
:10220000EE202AF491E0D90E9927E91EF91EB1CFEC
:1022100007C09FE7092FF92A9FEFD92EE92E0895CD
:10222000DD24EE24FF240027112708959F9299248E
:10223000AA24BB2488E1D216E306F40628F0D21AB9
:10224000E30AF40A089401C08894991CAA1CBB1CD8
:10225000DD0CEE1CFF1C8A9571F7D92CEA2CFB2CA7
:102260009F900895C8953196002008950E942910E6
:10227000E89488278A938A93D3DF11278D9180323F
:10228000E9F31197BBD098F08D3229F4109511968F
:102290008C91B4D060F08E3229F411968C91AED02E
:1022A00008F446C022960E94261081E008958C9181
:1022B000A5D0D8F547D01196D0F703958D919ED033
:1022C000E0F38E3229F48C9199D010F41196FBCF63
:1022D000853419F0853609F055C011968C918ED051
:1022E00060F08D3219F08B3221F0DCCF0880009441
:1022F000088211968C9182D0A8F68053898311961A
:102300008C917CD058F49981990F990F0980900D88
:10231000990F8053890F8983873220F689819881AC
:1023200099230AF48195080F2DC08E3289F61196F3
:102330008C9164D068F606D018F011960A95F8CF03
:102340001196C1CF4F2D3E2D2D2DDD0CEE1CFF1C07
:10235000A8F0DD0CEE1CFF1C88F0D20EE31EF41E6C
:1023600068F0DD0CEE1CFF1C48F0805309F0689407
:10237000D80E8827E81EF81E08F00895F42EE32EE4
:10238000D22E089534D019F116F5098308E921D029
:102390000695882787959F2D9F77980FF92E0150D6
:1023A000000F110F07958981882379F01AF4819520
:1023B000898306C0ECDE89818A958983D9F705C0B7
:1023C000F6DE89818A958983D9F72296089528DFD8
:1023D000FCCF0DD041F0FF2032F00A9531F0DD0C3A
:1023E000EE1CFF1CD2F788940895089408950024E9
:1023F0000D280E280F28002A00200895803320F091
:102400008A3310F4089408958894089591E005C0E3
:1024100092E003C094E001C098E024DF0D929A9509
:10242000E1F708957F930F93AF93BF938F939F939B
:102430008FB78F93E8948091AE0008E2081B21F4D7
:102440009CB10E94261013C00091AD00A4E8B0E03A
:1024500077279CB1A00FB71F9C93689483958093B6
:10246000AE000395083209F400270093AD009D30BB
:1024700011F40E949C0C8F918FBF9F918F91BF91FF
:10248000AF910F917F9118957F93AF93BF938F93E7
:102490009F938FB78F939091D900992399F09A9534
:1024A0009093D9009927AFEAB0E08091D700A80FA8
:1024B000B91F9C918395883209F488278093D700AF
:1024C0009CB901C055988F918FBF9F918F91BF91FB
:1024D000AF917F911895040F151F261F371F089580
:1024E000041B150B260B370B089504171507260739
:1024F00037070895000F111F221F331F08950095FD
:102500001095209530950F5F1F4F2F4F3F4F089527
:10251000019110810EC001911191219130810BC068
:102520000191108117FF05C03FEF2FEF04C000811C
:1025300011272227332737FF03C0E1DF8DE28D9378
:10254000CF93DF93CF92DF92EF92AA24BB24CC24C7
:10255000DD24EE2440E2CAE0DD2755E093E38881E4
:10256000890F87FD9F7083FD907F891B89935A9502
:10257000A9F7C0DFAA1CBB1CCC1CDD1CEE1C4A95B5
:1025800051F7E894EFE0FF2782910ED0EB30E0F7AF
:102590001EF068948A2D0CD088278D93EF90DF90E1
:1025A000CF90DF91CF910895982F829501D0892FF8
:1025B0008F70805D26F0803309F4089568948D93C0
:1025C000089500271127222733271DD08A3328F4A6
:1025D000803318F005D015D0F9CF0EF490CF0895C0
:1025E00080538F93402F512F622F732F83DF82DF11
:1025F00072DF80DF8F919927080F191F291F391F5C
:1026000008958D910895E894FCDF8032E9F38B32D0
:10261000D9F38930C9F38D3211F46894F2CF08955B
:1026200088278D93089594E081918D939A95E1F791
:10263000089581918D930A9519F08823D1F7089513
:10264000EFCF8FEF83959D919923E1F708956894DB
:1026500063F80895000000003A003D00323A313D31
:102660000000323A323D0000323A333D0000323A47
:10267000343D0000323A353D0000323A363D00002C
:10268000323A373D0000323A383D0000323A3131BB
:102690003D00574F4631303362002A0023303A4123
:1026A00044583D00210023303A4944473D0023303F
:1026B0003A49444E3D0023303A4241543D002330D4
:1026C0003A4552523D5B53796E746178204572727F
:0626D0006F725D210000A5
:00000001FF
